:10000000830100308A0061288C0003088301B70057
:100010003508B8009A30831281070B119A0B3528E6
:100020009A0A2E28051A35289A019A0A1B28051AB9
:100030002C2804309A009B0A35281B080A3A031919
:1000400026280310051A0314990C1928190898007A
:100050008D149A019A0A99019B0135281B080319EE
:100060001228013A031917281D289F080319492847
:100070001F080339031D48280D1D40280614412878
:10008000061083120D111E180D15031483129E0CF9
:100090009F031108031D9103FF30A207031CA30354
:1000A00023082204031D5928E130A2000130A300D7
:1000B0000D1483123808B500370883008C0E0C0E1F
:1000C00009000D3084000E306E200E308400353073
:1000D0006E208301812904068001840A0406031925
:1000E00000346B288207363434343234303482079B
:1000F0004F344934563483160514BA288312B1009C
:10010000861542298312AF008611422901308312DD
:1001100082200330CB288312AE008617CB208613B3
:10012000080083128D1C92288D1018080800831275
:10013000851083168510831208008312051083161C
:100140000510831208008316051485148312851088
:100150000510080083129D200130EC20972001300B
:10016000EC288312B1008900831608148312080852
:1001700008008316851401308312EC20972001308B
:10018000EC2883128620FA30CB201730AF000030E5
:10019000E020FA308B288312AF000A30910011085A
:1001A000031DCF28AF0BCD2808008312B0009F0895
:1001B000031DD7280D1130089E0034309F00080021
:1001C0008312B000E828B00A3003B1207E208312E9
:1001D000AF032F0FE32808008312B4008F00013013
:1001E000900000000000900BF1288F0BEF28080012
:1001F0008312B100AA2031082E217B200130EC208F
:1002000030082E217B2010298312AF000C29AF0A61
:100210002F03B120D5208312AE032E0F072908002B
:1002200083129D200130EC20831685140130831247
:10023000EC20831605140130EC288312AE012E0841
:10024000243E84000008AF002E08383E8312B021FF
:10025000AE0A08302E02031808001F298312B200CC
:10026000B301B21F362983160514382983129D2045
:100270008312B9200310B20DB30A083033020318F9
:10028000080031298312B2000F3086053208F03998
:100290008604061506110F308605320EF0398604E5
:1002A000061506110C30EC2001308605080083127B
:1002B000AC012C08383E8312B120B5002C08243E36
:1002C000840035088000AC0A08302C02031C592930
:1002D00097019C0117086C298312AE00243E84000C
:1002E0000008073992002E08243E840000081839BF
:1002F000B5000310B50C0310B50C0310350CA100AC
:100300000800831257213A225C22C12096218D1CBD
:100310008C2983129120AE220D1C87299608031D7B
:1003200087290D108312FF21262387298312AF010D
:1003300004302F0203189E2998309F29A830AE0060
:100340002F08243E84000008B0002E088312F820F5
:100350001430EC20AF0A08302F0203180800982947
:100360008312B00083168818B329831230088900DD
:100370002F08880003108B1B03148B13831608159A
:1003800055308900AA3089008814081103188B178A
:10039000831208008030831282205B307E20003080
:1003A0008A001D0877207E205D307E20AE0103305C
:1003B000AF001930E0202E08313E7E20AE0A053015
:1003C0002E0203180800D729F03083168600831206
:1003D0008614861506150608AD000611F030AD0529
:1003E00006150608AC0006112C0E0F39AD04831655
:1003F0008601831286100C30EC202D080800831231
:10040000AF011030AE000430AC00162A0F30860564
:100410002E0886040A30AD00AD0B0C2A0519182AE7
:10042000AF0A8519182AAF0A0310AE0DAC0B062AC5
:100430002F0808008312AE012E08303E8312B1202F
:10044000B5002E08243E840035088000AE0A08302E
:100450002E02031C1C2AAE012E08243E8400000834
:10046000AF002E08383EB021AE0A08302E02031825
:1004700008002C2A831206149F019A019A0A9B01F4
:1004800099018D1086131F30831685008601831213
:10049000A320E130A2000130A3000D100A30930028
:1004A0000230950006309400831681129A30831230
:1004B00081008B168B1708008312861086111E3060
:1004C000CB200F3086053030860406150611053026
:1004D000CB20061506110C30EC2006150611053050
:1004E000CB200F3086058616061506110C30EC2041
:1004F00028308220083082200C308220063082286A
:10050000C030831282204F307E200430170217083B
:1005100003188E2A313E7E204130912A2D3E7E20C6
:1005200042307E20AE010330AF001930E0201208C7
:10053000053A031D9D2A4D30A72A12082E06031DD9
:10054000A62A00308A0021087220A72A2E307E2099
:10055000AE0A05302E0203180800932A8312AD005C
:1005600064308B20A0080319D02A08300E020E0830
:100570000318C42A243E84002D0880008E0A3230DD
:100580008B202D08D5200E08083A031D0800A00175
:1005900096210230AE0017300421C12096010800D8
:1005A0002D08503A031DDB2A9601960A8E01A00100
:1005B000A00A2D08D5282D08523A031DFC2A9601C1
:1005C000960A2D08D520AC0108302C022C080318FF
:1005D000EC2A383EB120F02AF83E243E8400000880
:1005E000D52032308B20AC0A10302C02031CE42AB8
:1005F0000230AE00173004212D08573A031D0A2B94
:100600009601960A1D212D08D520C1200230AE008A
:10061000173004212D08433A031D162B2D08D52031
:100620001A22C1200230AE00173004212D083F3AB3
:10063000031D242B9601960A1730AE0000300421CA
:100640000230AE0017300421960108008312AC007E
:10065000063A031D332B1408063A031D312BAD0156
:10066000F02B0230402B1408063A031D3C2BAD0141
:10067000AD0A2C089400F02B93080319422B033089
:10068000AD00F02B0430402B0A3093009501950A01
:1006900008009601960A5C2B9C0183121D21C12043
:1006A0002A30D520960108008312962164308B20D1
:1006B0002D30D520960108002C0803194C2B013A47
:1006C0000319542B9C08031DB32B9C019C0A9D010C
:1006D000972B9D031D0FC02B02309D00C02B0330B4
:1006E0009D0A1D02031CC02B9D01C02B9703170FF1
:1006F000972B07309700972B9203120FC02B0530D2
:100700009200C02BA103210FC02B0330A100C02BEE
:100710001D080319762B013A03197C2B033A0319A0
:10072000822BC02B0830970A17020318970117086D
:1007300083126C21C02B0630920A1202031CC02BBC
:100740009201C02B0430A10A2102031CC02BA1017D
:10075000C02B1D080319922B013A03199B2B033A56
:100760000319A22BC02B2C08023A0319A92B013A1A
:100770000319882B073A03196F2B013A0319692BC8
:100780001708243E84001708B5000530B600031092
:10079000B50DB60BC72B3508B5002108B600031000
:1007A000B60D0310B60D0310360D3504120480008B
:1007B0008312CA218022960108000A309300950115
:1007C000950A0630940008009308031D930308005F
:1007D000950B0800023095000800063094000800D0
:1007E0002D080319442B013A0319492B033A031925
:1007F000DD2B013A0319E42B073A0319E82BED2B03
:02400E00F13F80
:104200004D0054005800200031002E0031002000E5
:1042100042002E00560045004C004C004500200096
:1042200028004300290032003000300033000D0028
:104230000A00200020002000200020002000200094
:10424000200020002000200020002000200020006E
:10425000200020002000200020002000200020005E
:104260001C003C005C007C001C003C005C007C00EE
:104270001C003C005C007C001C003C005C007C00DE
:00000001FF
